:10000000B6C0CFC0CEC0CDC0CCC0CBC0CAC0C9C0A6
:10001000C8C0C7C0C6C0C5C0C4C0C3C0C2C0C1C0BC
:10002000C0C0BFC0BEC00CC11FC135C186C485C41D
:100030006CC165C282C481C480C47FC47EC47DC4D7
:100040007CC47BC496C1FFC101C228C2AFC325C214
:10005000ACC300C412C4FEC310C40FC40EC42EC46B
:1000600047C140C16AC469C468C467C466C465C482
:1000700064C463C462C461C460C45FC45EC45DC45C
:100080002EC118C11AC159C41BC11DC128C12AC122
:100090001DC153C42AC151C450C42AC11AC11CC1B4
:1000A0001B5B306D1B5B324A1B5B303B3066004193
:1000B00076725573623530302D312E35207465726D
:1000C0006D696E616C206D6F64650D0A00456E741C
:1000D00065722053572056657273696F6E204D61AB
:1000E0006A6F7220696E20686578205B005D3A2037
:1000F00000456E7465722053572056657273696FA0
:100100006E204D696E6F7220696E20686578205B85
:10011000005D3A20000D0A4F4B2C206D792053577B
:100120002076657273696F6E206973206E6F773AFF
:1001300020002028686578290D0A005265616479DD
:100140002E204A75737420636C6F73652074686524
:10015000207465726D696E616C2E204E6F20726521
:10016000736574206E65656465642E0D0A00112444
:100170001FBECFE5D4E0DEBFCDBF10E0A0E6B0E00B
:10018000E4E9FFE002C005900D92AC36B107D9F763
:1001900011E0ACE6B0E001C01D92AF39B107E1F764
:1001A000ACC42ECFFF920F931F93CF93DF93182FE2
:1001B000EB01CB0101978D51914028F0C2E0D0E0D6
:1001C00080EC809376008BE144D59BE1F92E812F62
:1001D00040D5F1268D2F9927182F3BD5F1268C2F4E
:1001E00038D5FC268EE035D58EE0F8264ED6209701
:1001F00059F005E710E0F80180812BD5F8018191D5
:100200008F01F8262197B9F78F2D23D5E5E0CDB7DB
:10021000DEB78AC6A0E0B0E0EFE0F1E05FC6582E9E
:10022000E1E06E2E809175009927AA27BB27FC017B
:100230003197ED31F10508F080C3ED5EFF4F099471
:1002400081E0809375001092760088E080937700BB
:1002500089E0A8E7B0E0E1E6F0E001900D928A9530
:10026000E1F70BE010E06EC380917600883921F44D
:100270008091770023D50CC18E3929F480917700C5
:100280008093600005C18F3909F002C18091770029
:1002900080937400FDC0809176009927AA27BB2720
:1002A000FC01E058F040E032F10508F046C3E05DA3
:1002B000FF4F0994C0909D011DC0C0909E011AC0BF
:1002C00072E3C72E1BC069E1C62E18C032D5C82EF6
:1002D00011C0C09060000EC0C09074000BC052E00E
:1002E000C52E0CC041E0C42E09C03CE8C32E06C098
:1002F000CC2404C08FEFC81609F41FC303E010E03C
:1003000010927600C09277001DC3809176009927E5
:10031000AA27BB27B82FAA279927882720917700DB
:10032000332744275527A90133272227822B932BD4
:10033000A42BB52B20917800332744275527542F21
:10034000432F322F2227822B932BA42BB52B2091C6
:100350007900332744275527822B932BA42BB52BC9
:100360008093700090937100A0937200B09373001B
:100370008FC0A898FAD48091770099276AD502E0B7
:1003800010E080EC80937600EE24FF2480917900C9
:10039000813318F080E38093790080917A0088237C
:1003A00019F481E080937A00809179009927E8160A
:1003B000F90608F0C7C269D5A898809178009927F6
:1003C00048D50894E11CF11C80917D00E6D4809111
:1003D0007A0099273ED580917E00DFD480917A0003
:1003E000992737D5A89A80917F00D7D4C82E8091BD
:1003F0007A0099272ED580918000CFD4782E9091C5
:100400007C00933039F480917B00C81669F4109217
:1004100076000AC080917B00781611F41092760065
:10042000992311F49093760080917600882331F41B
:10043000A89880917900E82EFF24B6CF7ED484E17D
:1004400090E007D5B1CFFCD4A89A22C08091780063
:10045000A4D480917900A1D480917A009ED4809117
:100460007B009BD480917700882329F480917600CB
:100470009927EFD40DC0C6E9DC2E01C0DA9460E004
:1004800070E080E090EFC0D480FF02C0DD20B1F7C3
:1004900002E010E01092760055C266248824992468
:1004A0005401B6E9DB2E80917900843018F484E0A1
:1004B0008093790080917900813218F080E28093F6
:1004C00079008091700090917100A0917200B091BC
:1004D000730080936C0090936D00A0936E00B093B6
:1004E0006F00809176009927D82FCC2780917700D4
:1004F0009927C82BD92B91E0C931D90720F002E008
:1005000010E080EC1DC2C1D470907800CC24872DFF
:100510009927809590959C012170307080FF94C040
:10052000EE24FF24EC16FD0608F03AC105E710E0C2
:10053000662031F0E0FE04C080917A00886002C03D
:1005400080917A002AD4809170009091710050D4EB
:10055000F801828522D490917D00F8018285981758
:1005600099F08090700090907100A0907200B0900F
:1005700073008FEF9FEFA0E0B0E088229922AA22BB
:10058000BB227092780003C082E0809378007DD413
:10059000662019F482E090E05CD48091780099277D
:1005A00082FF19C0F6E9DF2E662031F0E0FE04C0BC
:1005B00080917C00886002C080917C00EED3C401F1
:1005C00017D480E0EAD3DA9490917D008917B9F4CA
:1005D000DD2051F714C083FF0EC0E6E9DE2E01C016
:1005E000DA9460E070E080E090EF0ED480FF07C006
:1005F000DD20B1F704C08091790099272AD46620C4
:1006000011F0E0FE13C08091700090917100A091F4
:100610007200B09173000196A11DB11D809370000E
:1006200090937100A0937200B0937300DD2011F4D9
:1006300070E8C72E0894E11CF11C0F5F1F4FEC16E9
:10064000FD0608F475CFACC079012C173D0708F002
:1006500053C005E710E019D4662031F0E0FE04C075
:1006600080917A00886002C080917A0096D3809150
:10067000700090917100BCD3F80182858ED3909167
:100680007D00F8018285981789F080907000909025
:100690007100A0907200B09073008FEF9FEFA0E008
:1006A000B0E088229922AA22BB2206C0809178005D
:1006B0008078806180937800662011F0E0FE13C09E
:1006C0008091700090917100A0917200B0917300C0
:1006D0000196A11DB11D8093700090937100A093AD
:1006E0007200B09373000894E11CF11C0F5F1F4F60
:1006F000EC16FD0608F4AFCFC8D38091780087FFD1
:100700004FC080917B0049D380916C0090916D0027
:100710006FD380E042D3662019F481E090E099D352
:1007200066E9D62E8091780085FF24C0811491045B
:10073000A104B104F9F0D501C40181709070A070DA
:10074000B070892B21F080917C00886002C080917C
:100750007C0023D3C4014CD380E01FD3DA94909162
:100760007D00891711F4DD2031F7DD20C9F450E850
:10077000C52E16C086FF10C001C0DA9460E070E09C
:1007800080E090EF41D380FF02C0DD20B1F7DD2093
:1007900039F441E8C42E04C080917900992759D3D7
:1007A00002E010E0C0927600CDC066248091760011
:1007B0009927D82FCC27809177009927C82BD92B40
:1007C000C090780091E0C931D90710F0C8E1D1E0BC
:1007D000EE24FF24EC16FD06A0F507E710E055D344
:1007E000662029F0E0FE03C08C2D886001C08C2DAE
:1007F000D4D28091700090917100FAD280E0CDD275
:10080000D8018C93662011F0E0FE13C08091700037
:1008100090917100A0917200B09173000196A11D9A
:10082000B11D8093700090937100A0937200B093FB
:1008300073000894E11CF11C0F5F1F4FEC16FD06BE
:1008400070F28E010D5F1F4F10927600CB58DF4F74
:100850001A8278C080917600A0D2809177009DD2D4
:10086000809178009AD28091790097D203E010E0CD
:10087000109276001092770065C007E710E0C0E0A4
:10088000D0E023E0D22EF80181918F0186D2C82ECC
:1008900080917600992721968C179D0711F4C092BC
:1008A000770085E090E0D5D2DA94D7FEECCF04E073
:1008B00010E0109276001092780044C0C09077004B
:1008C00070907800DD24CD2D80917600D81600F54B
:1008D00085E090E0BED2C71580F0DC1470F40D2DD9
:1008E00011270B581F4FEC2FFF27EB58FF4F848128
:1008F00054D2F8018283D39406C0EC2FFF27EB5823
:10090000FF4F84814AD2CF5F80917600C81700F3F1
:10091000DC1440F4ED2DFF27E958FF4F1192D394DA
:10092000DC14E0F3ED2DFF278F010D5F1F4F1092B8
:100930007600EB58FF4F128205C002E010E089EC10
:1009400080937600B801852D2DDCEFE0CDB7DEB7C2
:10095000E1C2EF92FF920F931F93CF93C1E0FC2E61
:10096000B2E0EB2E1FEF8111FE2C81E095D1C82F54
:100970008D30D1F18A30C1F10C2F00530A3038F09C
:100980008C2F8154863018F08052863020F51F3F1E
:1009900009F410E08C2F5DD10A3028F41295107FF5
:1009A0001C0F105317C08C2F8154212F33278630F2
:1009B00048F4A4E0220F331FAA95E1F71C2F120F71
:1009C000175308C0F4E0220F331FFA95E1F71C2FEC
:1009D000120F1755EA9481E05FD1C82F8D3021F0B6
:1009E0008A3011F0EE2041F6CD3011F0CA3009F412
:1009F000FA94FF2019F081E04FD1FACF812F992787
:100A0000CF911F910F91FF90EF9008958BE121D12D
:100A100085E41FD10895CF93C82F80EA90E02BD1B1
:100A20008FEA90E028D18DEC90E025D180919D0156
:100A300040E150E065E770E0992729D285E790E032
:100A40000CD18DEE90E017D18C2F83DF8F3F11F00A
:100A500080939D01DBDF81EF90E00DD180919E01BD
:100A600040E150E065E770E0992711D285E790E01A
:100A7000F4D081E191E0FFD08C2F6BDF8F3F11F03C
:100A800080939E01C3DFA1E0B0E080919E01082E1B
:100A900061D2A2E0B0E080919D01082E5BD2A0E07F
:100AA000B0E084E1082E56D285E191E0E4D0809157
:100AB0009D0140E150E065E770E09927E8D185E7C6
:100AC00090E0CBD08EE2C5D080919E01803110F4B1
:100AD00080E3BFD080919E0140E150E065E770E087
:100AE0009927D5D185E790E0B8D082E391E0C3D0D3
:100AF0008BE391E0C0D0CF910895CFE5D4E0DEBF85
:100B0000CDBFDD24BD2CCD2CC0E0D0E07E0198D03F
:100B1000B2D1A09AA89A789484E080939E0182E052
:100B200080939D01A0E0B0E00DD2802D843161F46E
:100B3000A1E0B0E007D2802D80939E01A2E0B0E05A
:100B400001D2802D80939D0181E0A6D004C080E079
:100B5000A3D0112321F58B3119F411E0082FF7CF21
:100B60008D3019F08A3009F065C02196BB2039F428
:100B70008A3029F49DE0D91611F401E0B02ED82E68
:100B8000BB2029F0C430D105F9F681E004C0C230A1
:100B9000D105D1F68B2D3FDFC0E0D0E0D5CF1130AD
:100BA00021F4C82E082712E0D2CF123031F40827E2
:100BB0009927F82EEE2413E0CACF133031F408271A
:100BC0009927E82AF92A14E0C2CF143041F4082703
:100BD0008E3009F0B9CF15E0C0E0D0E0B8CF1530C5
:100BE000A1F4CE15DF0534F591E0C831D90714F52D
:100BF0000827FE01EB58FF4F80832196A895CE155C
:100C0000DF0509F0A4CF16E0A2CF163099F48017C3
:100C100039F41E141F0424F4A8958C2DFBDA0AC0A5
:100C200080EB8093750081EC8093760062E070E049
:100C30008C2DB8DAEE24FF24DD24CD2CE70184CFFF
:100C400010BC81E090E089B988E18AB986E880BD6E
:100C500008955D9BFECF8CB90895CF93DF93EC018F
:100C60008881882329F08991F4DF88818823D9F746
:100C7000DF91CF910895CF93DF93EC01FC01219692
:100C80008491882331F0E5DFFE0121968491882349
:100C9000D1F7DF91CF910895CF93C82F5F9904C00A
:100CA000C111F3D05F9BFCCF8CB19927CF910895F0
:100CB0005F9B03C08CB15F99FDCF089510929C019A
:100CC000843048F081E080939C018CE080936A003E
:100CD0008CE090E00895833048F07098699A689AA3
:100CE00083E080936A0083E090E00895823048F0CA
:100CF0007098699A689882E080936A0082E090E038
:100D00000895813041F470986998689A80936A00D8
:100D100081E090E00895882341F47098689869987C
:100D200080936A0080E090E0089581E090E008956B
:100D3000089580916A00992708952DB11DB8C5982E
:100D40008CE590E0FC013197F1F7C59A0197F1F736
:100D5000C5982DB90895C29A8CE590E00197F1F7F6
:100D6000C29884E190E075D00895BA9AC29ABB9A6D
:100D7000C398BD9AC59884E190E06BD080919C01A6
:100D8000882329F481E58DB980916A0097DFC298A4
:100D900084E190E05ED0DFDF0895CF93DF93482FAA
:100DA00020E830E080919C01882331F44FB9779B93
:100DB000FECF8FB1992719C0C598ACE5B0E0C0E06F
:100DC000D0E0842F822311F0C39A01C0C398CD01D3
:100DD0000197F1F7B499322BC59ACD010197F1F73C
:100DE000C598269571F7832F9927DF91CF910895A4
:100DF0000F931F938C01812F9927CFDF802FCDDF99
:100E000099271F910F910895EF92FF920F931F93CF
:100E10007B018C01892F9927AA27BB27BEDFC80138
:100E2000AA27BB27BADFBB27A12F902F8F2DB5DFB5
:100E30008E2DB3DF99271F910F91FF90EF900895AA
:100E40001DB8C29ABB98C398BD98C598BA98C29865
:100E50000895CF93DF939C01892B51F0A4E7B3E071
:100E6000C0E0D0E0CD010197F1F721503040D1F73B
:100E7000DF91CF91089588E190E02FE00FB6F894CC
:100E8000A89581BD0FBE21BD0895A8950895FB01C9
:100E90009F0142306CF045325CF4642F772766D0B6
:100EA000805D8A330CF0895D8193CB010097A9F7AF
:100EB0001082C90100C0DC01FC0101900020E9F7AB
:100EC0003297AE17BF0730F47C9160817083319701
:100ED0006D93F7CF08952F923F924F925F926F924A
:100EE0007F928F929F92AF92BF92CF92DF92EF92BA
:100EF000FF920F931F93CF93DF93CDB7DEB7CA1B3B
:100F0000DB0B0FB6F894DEBF0FBECDBF09942A8865
:100F1000398848885F846E847D848C849B84AA840D
:100F2000B984C884DF80EE80FD800C811B81AA819A
:100F3000B981CE0FD11D0FB6F894DEBF0FBECDBF65
:100F4000ED010895E199FECFBFBBAEBBE09A1196CB
:100F50000DB20895E199FECFBFBBAEBB0DBA11969D
:100F60000FB6F894E29AE19A0FBE0895AA1BBB1B34
:100F700051E107C0AA1FBB1FA617B70710F0A61B99
:100F8000B70B881F991F5A95A9F780959095BC01BA
:040F9000CD010895F2
:0C0F9400014156524953505F32000100E9
:00000001FF
